:020000040800F2
:1000000000040020A102000851100008551000084B
:10001000A9100008551000087D100008A302000870
:10002000A3020008A3020008A3020008B5280008E4
:10003000A3020008A3020008A3020008A30200080C
:10004000A3020008A3020008A3020008A3020008FC
:10005000A3020008A3020008F93D0008253E00089D
:10006000513E00087D3E0008A93E0008A30200089A
:10007000A3020008A3020008A3020008A3020008CC
:10008000A3020008A3020008A3020008A3020008BC
:10009000A3020008A3020008A3020008D53E00083E
:1000A000A3020008A3020008A3020008A30200089C
:1000B000A3020008A3020008A3020008A30200088C
:1000C000A3020008A3020008A3020008A30200087C
:1000D000A3020008A3020008A3020008A30200086C
:1000E0003D3F0008A3020008A3020008A302000885
:1000F000A3020008A3020008A3020008A30200084C
:10010000A3020008A3020008793A0008A30200082D
:10011000A3020008A3020008A3020008A30200082B
:10012000A3020008A3020008A3020008A30200081B
:10013000A3020008A3020008A3020008A30200080B
:10014000A3020008A3020008A3020008A3020008FB
:10015000A3020008A3020008A3020008A3020008EB
:10016000A3020008A3020008A3020008A3020008DB
:10017000A3020008ED330008A3020008A302000850
:10018000A3020008A302000839110008A302000816
:10019000A3020008A3020008A3020008A3020008AB
:1001A000A3020008A3020008A3020008A30200089B
:1001B000A3020008A3020008A3020008A30200088B
:1001C000A3020008A3020008A3020008A30200087B
:1001D000A3020008D9330008A3020008A302000804
:1001E000A3020008A3020008A3020008A30200085B
:1001F000A3020008A3020008A3020008A30200084B
:10020000A3020008A3020008A3020008A30200083A
:10021000A3020008A3020008A3020008A30200082A
:10022000A3020008A3020008A3020008A30200081A
:10023000A3020008A3020008A3020008A30200080A
:10024000A3020008A3020008A3020008A3020008FA
:10025000A3020008A3020008A3020008A3020008EA
:10026000A3020008A3020008A3020008A3020008DA
:10027000A3020008A3020008A3020008A3020008CA
:10028000A3020008A3020008A3020008A3020008BA
:10029000A3020008A3020008A3020008A3020008AA
:1002A00002E000F000F8FEE772B6394880F30888F3
:1002B000384880F3098838484EF60851CEF20001DC
:1002C000086040F20000CCF200004EF63471CEF22D
:1002D00000010860BFF34F8FBFF36F8F40F2000043
:1002E000C0F2F0004EF68851CEF200010860BFF374
:1002F0004F8FBFF36F8F4FF00000E1EE100A4EF604
:100300003C71CEF200010860062080F31488BFF330
:100310006F8F02F00DFB03F02DFB4FF055301F499E
:100320001B4A91423CBF41F8040BFAE71C49194AA9
:1003300091423CBF41F8040BFAE71A491A4A1B4B99
:100340009A423EBF51F8040B42F8040BF8E7002034
:100350001749184A91423CBF41F8040BFAE702F0F2
:100360002BFB03F07BFB144C144DAC4203DA54F826
:10037000041B8847F9E700F03FF8114C114DAC42DF
:1003800003DA54F8041B8847F9E702F013BB0000B6
:1003900000040020002400200000000800000020CD
:1003A00000040020A0430008002400204424002072
:1003B0004824002060350020A0020008A0020008A8
:1003C000A0020008A00200082DE9F04F2DED108AD0
:1003D000C1F80CD0D0F80CD0BDEC108ABDE8F08F7D
:1003E000002383F311882846A047002001F0CAFEAD
:1003F00001F07AFE00DFFEE738B5204C6FF07403A1
:10040000002523701E236570A570E5702571657148
:10041000A571E57125726572A372E57200F030FD79
:1004200020B10E2325726572A372E57202F004FA00
:10043000044602F039FA0546D8B9114B9C421AD04D
:1004400001339C4218BF054641F2883404BF0125A0
:100450000024002002F0FAF90DB100F0B7F800F026
:100460009DFD00F063FC204600F070F900F0AEF84E
:10047000F9E70024EDE70446EBE700BF482400203D
:10048000010007B008B500F0CFFBA0F120035842EF
:10049000584108BD07B5054B02211B88ADF8043053
:1004A00001A800F02DFC03B05DF804FB44400008F7
:1004B000064991F8243033B100230822086A81F8F4
:1004C000243000F057BC0120704700BF6824002092
:1004D0002DE9F84F234C94F82430054688461746FA
:1004E0008BBB2E46DFF87C90002F38D094F824A0E8
:1004F000BAF1000F05D12022FF214846266200F004
:100500003BFDCAF10805BD4228BF3D465FFA85FBA9
:10051000AD0041462A4604EB8A0000F003FD94F842
:100520002430A7EB0B079B445FFA8BFBBBF1080F52
:100530002E44A844FFB284F824B0D5D1FFF7B8FF09
:100540000028D1D108E0266A06EB8306B042C9D064
:10055000FFF7AEFF0028C4D10020BDE8F88F0120CE
:10056000BDE8F88F6824002010B5202383F311889C
:100570001248C3680BB101F08BFE0023104A0F48EC
:100580004FF47A7101F048FE002383F311880D4C7B
:10059000236813B12368013B2360636813B1636868
:1005A000013B6360084B1B7833B9636823B90220B1
:1005B00000F0A6FC3223636010BD00BF542400206D
:1005C0006905000898250020902400202DE9F041BD
:1005D000544B554953F8042F013201D1BDE8F08145
:1005E0008B42F7D1514C524B22689A4240F298808C
:1005F000504B9B6803F1006303F500339A4280F08F
:100600008F80002000F0AEFB4B4B0220187000F0F2
:100610006BFC4A4BD3F8E8200022C3F8E820D3F85B
:100620001011C3F81021D3F81011D3F8EC10C3F84F
:10063000EC20D3F81411C3F81421D3F81411D3F813
:10064000F010C3F8F020D3F81811C3F81821D3F82C
:100650001811D3F8801041F00061C3F88010D3F86E
:10066000801021F00061C3F88010D3F88010D3F817
:10067000801041F00071C3F88010D3F8801021F091
:100680000071C3F88010D3F8803072B62C492D4B1E
:100690000B601D682468BFF34F8FBFF36F8F2A4B29
:1006A000C3F88420BFF34F8F5A6922F480325A6115
:1006B000BFF34F8FD3F88020C2F3C906C2F34E3286
:1006C0005201B70743F6E07E02EA0E08384631468B
:1006D000013948EA000CB1F1FF3FC3F874C200F1E0
:1006E0004040F5D1203A12F1200FEDD1BFF34F8FEA
:1006F000BFF36F8FBFF34F8FBFF36F8F5A6922F431
:1007000000325A610022C3F85022BFF34F8FBFF36B
:100710006F8F202383F31188AD4685F30888204727
:10072000BDE8F081FCFF01081C000208040002087B
:10073000FFFF0108482400209024002000440258B4
:1007400008ED00E00000020800ED00E02DE9F04FA8
:10075000BA4C97B020228246FF210EA8A66800F06E
:100760000BFCB74A1378A346A3B9B6480121C3606E
:100770001170202383F31188C3680BB101F088FD49
:100780000023B14AAF484FF47A7101F045FD0023D0
:1007900083F31188BAF1000F02D0AC4BC3F800A06C
:1007A000AB4BAA4A00241C70546025462746984645
:1007B000012000F099FBBAF1000F00F0FA81A34B81
:1007C0001B68002B40F0F58117B0BDE8F08F0220C8
:1007D000FFF758FE002840F0E6819E4B1B88ADF8DD
:1007E0002430022109A800F08BFAE1E74FF47A7077
:1007F00000F01AFA031E0193EFDB0220FFF742FE1E
:1008000081460028E9D0019B581E042800F2CD81C2
:10081000DFE800F0030D1013160016A8052340F8BA
:10082000343D042100F06CFA4C46002752E00421CC
:100830008248F7E704218848F4E704218748F1E774
:100840001C24204600F090FA04340990042109A8E1
:1008500000F056FA2C2CF4D1E6E7002DBDD0002C88
:10086000BBD00220FFF70EFE0546002800F09F8156
:10087000012000F077FA022088F8000000F034FB35
:100880000024E3B21846019300F07CFA814648B197
:10089000019B184600F086FA01340028F1D12C465D
:1008A0006F4B9BE70123022088F8003000F00EFB1D
:1008B0004E46DBF808309E4206D2304600F054FA2D
:1008C0000130ECD10436F4E7604B002688F8006074
:1008D0005E602C4600F058FB1DB1002C18BF4FF095
:1008E000000AFFF7D7FD63E7002D3FF476AF002C39
:1008F0003FF473AF022088F8000000F0F5FA3220D0
:1009000000F092F9B0F10009C0F2518119F003052D
:1009100040F04D81DBF8082006EB0903934200F21A
:100920004681B9F5807F00F242814D450DDA4FF4E2
:100930007A7000F079F90290029B002BC0F23781A7
:10094000484A029BAB540135EFE7C820FFF79AFDF8
:100950000546002800F02B811F2E11D8C6F1200477
:100960004C4528BF4C460EAB26F0030022463D49BD
:10097000184400F0D7FA2246FF213A4800F0FCFA6A
:100980004FEAA9095FFA89F236493046FFF7A0FD20
:100990000446002883D006EB890605469AE7022024
:1009A000FFF770FD00283FF418AFFFF781FD002826
:1009B0003FF413AF4FF000094B46DBF80820914598
:1009C0001CD2B9F11F0F12D80E9A01320FD029F0A4
:1009D000030216A90A4452F8202C09921846042250
:1009E00009A900F075FB09F104090346E5E748464B
:1009F000019300F0B9F9019B0990EFE716A80421D3
:100A000040F84C3D00F07CF964E716A8002340F85C
:100A1000343D642100F040F900287FF4DEAE02206E
:100A2000FFF730FD00283FF4D8AE099800F0CCF96C
:100A300016AB43F8480D04211846E3E7482400208C
:100A400094250020542400206905000898250020E2
:100A500090240020464000084C2400205024002010
:100A6000484000089424002016A8002340F8343D94
:100A7000642100F011F900287FF4AFAE0220FFF7E7
:100A800001FD00283FF4A9AE099800F09FF916ABCC
:100A900043F8440DCFE70220FFF7F4FC00283FF4B1
:100AA0009CAE00F099F916AB43F8400DC3E7022065
:100AB000FFF7E8FC00283FF490AE09A9142000F0ED
:100AC00091F9814616A8042140F83C9D00F018F9E0
:100AD000494609A896E7322000F0A6F8B0F10009CF
:100AE000FFF67BAE19F0030F7FF477AEDBF808203A
:100AF00009EB070393423FF670AE0220FFF7C2FCFA
:100B000000283FF46AAE29F00309B9444F453FF489
:100B1000E1AE384600F028F90421089008A800F05A
:100B2000EFF80437F2E74FF47A70FFF7ABFC0028D8
:100B30003FF453AEFFF7BCFC00283FF4B1AE0E9B70
:100B400001330CD008220EA90020FFF7C1FC0028B9
:100B50003FF4A6AE2022FF210EA800F00DFAFFF709
:100B600099FC304801F014FB2EE616A8002340F84B
:100B7000343D642100F090F8814600287FF42DAECA
:100B80000220FFF77FFC00283FF427AEFFF782FC2E
:100B900041F2883001F0FCFA099800F039FACA46AF
:100BA00000F0F2F904E6054694E6002715E625462E
:100BB00013E6002000F038F80290029B002BFFF6AD
:100BC000FAAD012000F082F9029B213B122B3FF687
:100BD000EFAD01A252F823F0CF070008ED0700089F
:100BE0005B080008B1070008B1070008B10700085A
:100BF000E9080008D70A00089F0900080B0A000846
:100C0000690A0008970A0008B1070008AF0A00083F
:100C1000B1070008270B0008D5080008B107000835
:100C20006B0B0008A08601002DE9F34702AE0024FB
:100C30004FF47A7506F8014D144FDFF8588045439C
:100C400097F900305A1C5FFA84F901D0A34212D1FF
:100C500058F8240003680122D3F820A031462B461F
:100C6000D047012807D10A4B9DF8070083F8009070
:100C700002B0BDE8F0870134022CE1D14FF4FA70E4
:100C800001F086FA4FF0FF30F2E700BF00240020A9
:100C9000BC2500205C4000082DE9F0474FF47A7530
:100CA000144FDFF8588006464D43002497F9003072
:100CB0005A1C5FFA84F901D0A34210D158F82400DD
:100CC00003680422D3F820A031462B46D0470428DD
:100CD00005D1094B83F800900020BDE8F08701346E
:100CE000022CE3D14FF4FA7001F052FA4FF0FF30CA
:100CF000BDE8F08700240020BC2500205C400008EF
:100D000030B4074B1A78074B53F822402368DD694B
:100D1000054B0A46AC460146204630BC604700BF42
:100D2000BC2500205C400008A0860100F8B501F059
:100D300075FC094C094E0A4F207000253068237855
:100D4000834207D901F066FC336805440133BD4294
:100D50003360F3D9F8BD00BFBD250020A0250020D9
:100D6000FFFF010001F01CBD00F1006000F5003044
:100D70000068704700F10060920000F5003001F05B
:100D8000A9BC0000054B1A68054B1B789B1A8342CF
:100D900002D9104401F03EBC00207047A02500207D
:100DA000BD25002038B5074D04462868204401F0D1
:100DB00037FC28B928682044BDE8384001F042BC1F
:100DC00038BD00BFA025002000207047014BC0584F
:100DD000704700BF00E8F11F014B1868704700BF63
:100DE0000010005CF0B5244B244C1B682788656814
:100DF00094F90820C3F30B06BE424FEA134328D0F0
:100E0000A789BE4206D101220C2505FB0244656874
:100E100094F9082041F20104A3421CD041F20304DA
:100E2000A3421AD042F20104A34218D042F20304B2
:100E3000A34208BF5622441E0C44013D0B46A34268
:100E400017D215F9016F581C5EB1034600F8016C0A
:100E5000F5E70022D8E75A22EDE75922EBE75822BE
:100E6000E9E72C2584421D7001D9981C5A70401A5C
:100E7000F0BD1846FBE700BF0010005C0424002012
:100E8000104B5B8841F201018B429AB211D041F2C2
:100E900003018B420FD042F201039A420DD042F27D
:100EA00003039A420BD10323074A02EB8303D8784A
:100EB00070470023F8E70123F6E70223F4E7002058
:100EC000704700BF0010005C4C400008022804D1AD
:100ED0004FF40002034B9A6170470128FCD14FF494
:100EE0008002F7E700080258022803D18022034B52
:100EF0009A6170470128FCD14022F8E700080258A7
:100F0000022805D1064A536983F080035361704774
:100F10000128FCD1024A536983F04003F6E700BF81
:100F20000008025810B50023934203D0CC5CC4548F
:100F30000133F9E710BD000030B5441E14F9010F6C
:100F40000B4660B193F90050854201F1010106D1D1
:100F50001AB993F90020801A30BD013AEEE7002A51
:100F6000F7D1104630BD000002460346981A13F927
:100F7000011B0029FAD1704702440346934202D074
:100F800003F8011BFAE77047024B1A78024B1A70FC
:100F9000704700BFBC2500200024002038B5164C47
:100FA000164D204600F026FC2946204600F04EFC57
:100FB0002D681348D5F89020D2F8043843F0020386
:100FC000C2F8043801F0E4F80E49284600F04EFD5E
:100FD000D5F890200C48D2F804380C4923F00203CD
:100FE000C2F80438A0424FF4E1330B6003D0BDE8EF
:100FF000384000F05DBB38BDEC2A00203C410008C1
:1010000040420F006441000840260020A425002033
:1010100038B50B4B1A780B4B53F822400A4B9C42C5
:1010200005460CD0094B002118461822FFF7A4FFF3
:10103000056001462046BDE8384000F039BB38BDA8
:10104000BC2500205C400008EC2A0020A4250020DC
:10105000FEE7000000B59BB0EFF309816822684607
:10106000FFF760FFEFF30583034B9A6B9A6A9A6A66
:101070009A6A9A6A9B6AFEE700ED00E000B59BB0B1
:10108000EFF3098168226846FFF74CFFEFF3058311
:10109000044B9A6B9A6A9A6A9A6A9A6A9A6A9B6AE3
:1010A000FEE700BF00ED00E000B59BB0EFF3098163
:1010B00068226846FFF736FFEFF30583034B5A6B50
:1010C0009A6A9A6A9A6A9A6A9B6AFEE700ED00E059
:1010D00030B5084D0A4491420BD011F8013B092468
:1010E0005840013CF7D040F300032B4083EA500006
:1010F000F7E730BD2083B8ED002304491A465A5063
:10110000C8180833802B4260F9D17047C0250020F1
:10111000024A136843F0C003136070470078004030
:10112000044B5A6810439A6858600AB1181D10475A
:10113000704700BF402600202DE9F84F404EF56D66
:101140002F68EC692C62210718D014F0080F0CBF2F
:1011500000208020E20748BF40F02000A30748BFDE
:1011600040F04000610748BF40F48070202383F3C3
:101170001188FFF7D5FF002383F31188E20509D515
:10118000202383F311884FF40070FFF7C9FF002379
:1011900083F31188DFF8A8A04FF020094FF0000B6F
:1011A00014F0200832D13B0615D5DFF898A04FF097
:1011B000200920060FD589F31188504600F0ECF97C
:1011C000002830DA0820FFF7ABFF27F080032B6000
:1011D000002383F3118879060DD562060BD52023F1
:1011E00083F31188F26C336D9A4201D1336C03BBE7
:1011F000002383F31188E30604D5B26E13690BB1A3
:1012000050699847BDE8F84F01F064BB89F3118835
:10121000AB8C96F864105046194000F057FA8BF3E7
:101220001188EC69BCE780B2288588F31188EC69E5
:10123000BFE7102027F04007FFF772FF2F60D7E7C6
:10124000402600207826002013B5104C204600F0E0
:1012500023FA04F11400009400234FF400720C49A7
:1012600000F0E4F804F1380000940A4B0A494FF406
:10127000007200F05DF9094BE365094B23660C2110
:10128000522002B0BDE8104000F05EB840260020B9
:10129000AC26002011110008AC2800200078004086
:1012A00000E1F505254B002908BF1946037C81663E
:1012B000012B30B511D1224B98420ED1214BD3F8DE
:1012C000E82042F08042C3F8E820D3F8102142F031
:1012D0008042C3F81021D3F810310A68036EC46D40
:1012E00003EB5203B3FBF2F34A68150442BF23F049
:1012F000070503F0070343EA4503E3608B6843F007
:1013000040036360CB6843F00103A36042F496732B
:1013100043F00103236051054FF0FF33236205D5ED
:1013200012F0102205D0B2F1805F04D080F8643052
:1013300030BD7F23FAE73F23F8E700BF8040000875
:10134000402600200044025800F1604300F01F02D4
:10135000400903F5614309018000C9B200F1604012
:1013600083F8001300F5614001239340C0F88031F9
:1013700003607047F8B5154682680669AA420B46B5
:10138000816938BF8568761AB542044607D2184687
:101390002A46FFF7C7FDA3692B44A3610DE011D9CD
:1013A00032461846FFF7BEFDAF1B3A46E1683044AF
:1013B000FFF7B8FDE2683A44A261A3685B1BA36033
:1013C0002846F8BD18462A46FFF7ACFDE368E4E777
:1013D00083682DE9F041044693421546266938BFDB
:1013E00085684069361AB5420F4606D22A46FFF78D
:1013F00099FD63692B4463610DE012D93246A5EB78
:101400000608FFF78FFD4246B919E068FFF78AFD2D
:10141000E26842446261A3685B1BA3602846BDE8A2
:10142000F0812A46FFF77EFDE368E4E710B50A4441
:101430000024C361029B006040608460C1608161E0
:1014400041610261036210BD08B58269436993423C
:1014500001D1826882B98268013282605A1C42617D
:101460001970426903699A4201D3C368436100213C
:1014700000F0AAFE002008BD4FF0FF3008BD0000BC
:1014800070B5202304460E4683F31188A568A5B1E4
:10149000A368A269013BA360531CA361157822696C
:1014A000934224BFE368A361E3690BB120469847E8
:1014B000002383F31188284670BD3146204600F092
:1014C00073FE0028E2DA85F3118870BD2DE9F74F2D
:1014D00005460F4690469A46D0F81C90202686F383
:1014E00011884FF0000B144664B122463946284655
:1014F000FFF740FF034668B95146284600F054FE06
:101500000028F1D0002383F31188A8EB040003B076
:10151000BDE8F08FB9F1000F03D001902846C8470D
:10152000019B8BF31188E41A1F4486F31188DBE7D3
:10153000C16081614161C3611144009B00604060F2
:101540008260016103627047F8B504460E46174693
:10155000202383F31188A568A5B1A368013BA3608C
:1015600063695A1C62611E70236962699A4224BFD2
:10157000E3686361E3690BB120469847002080F37C
:101580001188F8BD3946204600F00EFE0028E2DA48
:1015900085F31188F8BD0000836942699A4210B54D
:1015A00001D182687AB98268013282605A1C8261F4
:1015B0001C7803699A4201D3C3688361002100F05B
:1015C00003FE204610BD4FF0FF3010BD2DE9F74F50
:1015D00005460F4690469A46D0F81C90202686F382
:1015E00011884FF0000B144664B122463946284654
:1015F000FFF7EEFE034668B95146284600F0D4FDD9
:101600000028F1D0002383F31188A8EB040003B075
:10161000BDE8F08FB9F1000F03D001902846C8470C
:10162000019B8BF31188E41A1F4486F31188DBE7D2
:10163000026843681143016003B118477047000016
:101640001430FFF743BF00004FF0FF331430FFF7B3
:101650003DBF00003830FFF7B9BF00004FF0FF3347
:101660003830FFF7B3BF00001430FFF709BF0000A8
:101670004FF0FF311430FFF703BF00003830FFF7A1
:1016800063BF00004FF0FF323830FFF75DBF00004E
:1016900000207047FFF7D8BD044B03600023436070
:1016A0008360C36001230374704700BF9840000843
:1016B00010B52023044683F31188FFF7F3FD0223BE
:1016C0002374002383F3118810BD000038B5C3696B
:1016D00004460D461BB904210844FFF7A9FF29461B
:1016E00004F11400FFF7B0FE002806DA201D4FF4C5
:1016F0008061BDE83840FFF79BBF38BD0268436892
:101700001143016003B118477047000013B5446BE3
:10171000D4F894341A681178042915D1217C02294F
:1017200012D11979128901238B4013420CD101A9DE
:1017300004F14C0001F08CFFD4F89444019B217912
:101740000246206800F0EAF902B010BD143001F042
:101750000FBF00004FF0FF33143001F009BF00004D
:101760004C3001F0E1BF00004FF0FF334C3001F08E
:10177000DBBF0000143001F0DDBE00004FF0FF3190
:10178000143001F0D7BE00004C3001F0ADBF0000B6
:101790004FF0FF324C3001F0A7BF0000D0F8942486
:1017A00038B5136819780429054601D0012038BDE1
:1017B000017C0229FAD112795C8901209040044011
:1017C000F4D105F1140001F06FFE02460028EDD0BF
:1017D000D5F894544FF480732868697900F08CF937
:1017E000204638BD406BFFF7D9BF0000002070478E
:1017F000704700007FB5124B036000234360836095
:10180000C360012502260F4B057404460290019324
:1018100000F18402294600964FF48073143001F0E1
:101820001FFE094B0193029400964FF4807304F558
:101830002372294604F14C0001F0E6FE04B070BDAD
:10184000C0400008E51700080D1700080A682023AB
:1018500083F311880B790B3342F823004B79133350
:1018600042F823008B7913B10B3342F82300022393
:101870000374C0F89414002383F3118870470000A8
:1018800038B5037F044613B190F85430ABB9201D2E
:1018900001250221FFF732FF04F1140025776FF0D4
:1018A000010100F09DFC84F8545004F14C006FF0ED
:1018B0000101BDE8384000F093BC38BD10B50121EE
:1018C00004460430FFF71AFF0023237784F85430CE
:1018D00010BD000038B504460025143001F0D8FDD5
:1018E00004F14C00257701F0A7FE201D84F8545028
:1018F0000121FFF703FF2046BDE83840FFF74EBF48
:1019000090F8803003F06003202B19D190F88120EB
:10191000212A0AD0222A4FF000030ED0202A0FD10C
:10192000084A42670722826704E0064B43670723A1
:1019300083670023C3670120704743678367F9E724
:10194000002070471C240020D0F8943437B51A6862
:101950001178042904461AD1017C022917D119797A
:10196000128901238B40134211D100F14C05284606
:1019700001F022FF58B101A9284601F069FED4F810
:101980009444019B21790246206800F0C7F803B017
:1019900030BD000001F10B03F7B550F823400546B8
:1019A0000E46F4B1202383F3118805EB8607201D32
:1019B0000821FFF7A3FEFB685B691B684C3413B179
:1019C000204601F053FE01A9204601F041FE0246E7
:1019D00048B1019B3146284600F0A0F8002383F36C
:1019E000118803B0F0BDFB685A691268002AF5D06F
:1019F0001B8A013B1340F1D105F18002EAE70000A8
:101A0000133138B550F82140DCB1202383F311881D
:101A1000D4F894241368527903EB8203DB689B6942
:101A20005D6845B104216018FFF768FE294604F19E
:101A3000140001F043FD2046FFF7B0FE002383F3BE
:101A4000118838BD7047000001F03EB801230370D3
:101A50000023436000F1300200F1500142F8043BE2
:101A60008A42D361FAD103814381704738B5044675
:101A7000202383F311880025416000F10C0300F15D
:101A8000300243F8045B9342FBD1204601F03EF85C
:101A90000223237085F3118838BD000070B500EB78
:101AA000810305465069DA600E46144618B11022CB
:101AB0000021FFF761FAA06918B110220021FFF799
:101AC0005BFA31462846BDE8704001F031B90000AC
:101AD000038903F001030381438903F00103438178
:101AE00000F1300200F11003002143F8041B93427F
:101AF000FBD101F0B5B90000F0B400EB81044789D7
:101B0000E4680125A4698D403D434581236000239D
:101B1000A2606360F0BC01F0D1B90000F0B400EB4A
:101B200081040789E468012564698D403D4305818E
:101B300023600023A2606360F0BC01F049BA00009A
:101B4000022310B5037000230446A0F8883080F803
:101B50008A3080F88B300381438100F10C0200F160
:101B6000300142F8043B8A42FBD184F870302046B1
:101B700001F072F863681B6823B120460021BDE8BC
:101B80001040184710BD0000436802781B6880F8B9
:101B90008C20052202700BB1042118477047000009
:101BA000436890F88C201B6802700BB10521184720
:101BB0007047000090F8703070B5044613B10023F0
:101BC00080F8703004F18002204601F06DF96368FE
:101BD0009B6863BB94F8805015F0600615D194F8AB
:101BE000813005F07F0545EA032540F202339D422E
:101BF00000F00E815BD8022D00F0DC803FD8002D74
:101C000000F08780012D00F0CF800021204601F0F8
:101C100003FC0021204601F0F3FB63681B6813B14D
:101C2000062120469847062384F8703070BD204670
:101C300098470028CED094F8872094F8863043EA5D
:101C40000223A26F934238BFA36794F98030A56F37
:101C5000002B4FF0200380F2FD80002D00F0EC807F
:101C6000092284F8702083F311880021A36F626F2A
:101C70002046FFF753FF002383F3118870BDB5F5AD
:101C8000817F00F0B180B5F5407F49D0B5F5807F08
:101C9000BBD194F88230012BB7D1B4F8883023F04F
:101CA0000203A4F888306667A667E667C3E740F2D8
:101CB00001639D421ED8B5F5C06F3BD2B5F5A06F4C
:101CC000A3D1B4F88030B3F5A06F0ED194F8823070
:101CD00084F88A30204601F01DF863681B6813B150
:101CE0000121204698470323237000236367A367DD
:101CF000E367A0E7B5F5106F32D040F602439D428E
:101D000052D0B5F5006F80D104F18B0363670123D6
:101D100024E004F1880363670223A367E5678AE789
:101D200094F88230012B7FF470AFB4F8883043F020
:101D30000203B6E794F88520616894F884304D6812
:101D400094F8831043EA0223204694F88220A8479F
:101D500000283FF45AAF436863670368A367A4E7AA
:101D60002378042B10D1202383F311882046FFF71A
:101D7000AFFE86F31188636884F88B601B680321CB
:101D800021700BB12046984794F88230002BACD0DC
:101D900084F88B300423237063681B68002BA4D065
:101DA000022120469847A0E7374B63670223A367C9
:101DB00000239DE794F8841011F0800F204601F075
:101DC0000F010ED001F062F8012806D002287FF43E
:101DD0001CAF2E4B6367A06767E72D4B6367A56752
:101DE00063E701F045F8EFE794F88230002B7FF4C9
:101DF0000CAF94F8843013F00F013FF476AF1A065D
:101E0000204602D501F020FB6FE701F011FB6CE7E3
:101E100094F88230002B7FF4F8AE94F8843013F0FD
:101E20000F013FF462AF1B06204602D501F0F4FA21
:101E30005BE701F0E5FA58E7142284F8702083F399
:101E400011882B462A4629462046FFF755FE85F382
:101E5000118870BD5DB1152284F8702083F311885C
:101E60000021A36F626F2046FFF746FE03E70B22B7
:101E700084F8702083F311882B462A462946204691
:101E8000FFF74CFEE3E700BFF0400008E840000821
:101E9000EC40000838B590F870300446152B29D86E
:101EA000DFE803F03E28282828283E28280B293977
:101EB00028282828282828283E3E90F8871090F8BF
:101EC0008620836F42EA01229A4214D9C268128A9C
:101ED000B3FBF2F502FB15356DB9202383F31188AE
:101EE0002B462A462946FFF719FE85F311880A2357
:101EF00084F8703038BD142384F87030202383F3C5
:101F0000118800231A4619462046FFF7F5FD0023E5
:101F100083F3118838BDC36F03B198470023E7E707
:101F2000002101F079FA0021204601F069FA636886
:101F30001B6813B10621204698470623D8E7000006
:101F400090F87020152A38B5044622D80123934012
:101F500040F6416213421DD113F480150FD19B024C
:101F600017D50B2380F87030202383F311882B467C
:101F70002A462946FFF7D2FD85F3118838BDC3688C
:101F80009B695B682BB9C36F03B19847002384F842
:101F9000703038BD002101F03FFA0021204601F0E9
:101FA0002FFA63681B6813B1062120469847062361
:101FB000EDE70000024B00221B605B609A607047F7
:101FC000AC2A0020002303748268054B1B689968C3
:101FD0009142FBD25A6803604260106058607047BB
:101FE000AC2A002008B5202383F31188037C032B3F
:101FF00005D0042B0DD02BB983F3118808BD43699C
:1020000000221A604FF0FF334361FFF7DBFF00232C
:10201000F2E790E80C001A6002685360F2E70000F3
:10202000002303748268054B1B6899689142FBD8B2
:102030005A6803604260106058607047AC2A002004
:10204000054B19690874186802681A6053601861B2
:1020500001230374FEF7B8B9AC2A002030B54B1C3D
:1020600087B005460A4C10D023690A4A01A800F03F
:10207000D3F82846FFF7E4FF049B13B101A800F052
:1020800007F92369586907B030BDFFF7D9FFF8E7B2
:10209000AC2A0020E51F000838B50C4D41612B69C2
:1020A00081689A689142044603D8BDE83840FFF73A
:1020B00089BF1846FFF786FF01232C610146237470
:1020C0002046BDE83840FEF77FB900BFAC2A0020AB
:1020D000044B1A681B6990689B68984294BF002063
:1020E00001207047AC2A002010B5084C23682069F5
:1020F0001A6822605460012223611A74FFF790FF6E
:1021000001462069BDE81040FEF75EB9AC2A002008
:102110008260022202740022427470478368A3F135
:102120007C0243F80C2C026943F83C2C426943F8CA
:10213000382C074A43F81C2CC26843F8102C0222A2
:1021400003F8082C002203F8072CA3F118007047AD
:10215000E103000810B5202383F31188FFF7DEFFA9
:1021600000210446FFF798FF002383F311882046DF
:1021700010BD0000024B1B6958610F20FFF760BFC4
:10218000AC2A0020202383F31188FFF7F3BF00005F
:1021900008B50146202383F311880820FFF75EFF6E
:1021A000002383F3118808BD49B1064B42681B69BF
:1021B00018605A60136043600420FFF74FBF4FF070
:1021C000FF307047AC2A00200368984206D01A6896
:1021D0000260506059611846FFF7F4BE7047000076
:1021E00038B504460D462068844200D138BD0368E6
:1021F00023605C604561FFF7E5FEF4E7054B03F102
:1022000014025A619A614FF0FF32DA6100221A62B9
:10221000704700BFAC2A0020F8B503611A4BC260BA
:102220005C6A1A4B1A46022952F8145F38BF022121
:10223000954206461F460AD1586198611C620560A6
:10224000456081600819BDE8F84001F0D7BA186A06
:10225000AB68241A0C1902D3E41A2D6804E09C42DE
:1022600002D2204401F0DAFAAB689C42F4D86B68E1
:10227000736035601E606E60B460A9684FF0FF3314
:10228000091BA960FB61F8BD000C0040AC2A0020CE
:1022900010B41A4C234653F8141F814210D04168E1
:1022A00002680A60026851609A424FF00001C16002
:1022B00003D0936881680B4493605DF8044B7047CA
:1022C0000A68626100209A425360C86003D15DF8D9
:1022D000044B01F09DBA9368886803449360084AF0
:1022E000206A526A121A9342E7D9991A012998BFB3
:1022F000931C18445DF8044B01F090BAAC2A0020FE
:10230000000C004000207047FEE70000704700000E
:102310004FF0FF3070470000022906D0032906D095
:102320000129064818BF0020704705487047032A56
:102330009ABF044800EBC20000207047C04100086B
:10234000744100082424002070B59AB001AD0646FF
:1023500008462946144600F095F82846FEF704FE84
:10236000C0B2431C5B0086E818002370032363702F
:10237000002302341946DAB2904204F1020401D873
:102380001AB070BDEA5C04F8022C04F8011C013399
:10239000F1E7000008B5202383F311880348FFF715
:1023A000D3FA002383F3118808BD00BFEC2A002074
:1023B00010B50446052916D8DFE801F016150316F6
:1023C000161D202383F311880E4A0121FFF766FBB7
:1023D00020460D4A0221FFF761FB0C48FFF77AFA0D
:1023E000002383F3118810BD202383F3118807484D
:1023F000FFF746FAF4E7202383F311880348FFF739
:102400005DFAEDE7F440000818410008EC2A0020CE
:1024100038B50C4D0C4C0D492A4604F10800FFF765
:1024200093FF05F1CA0204F110000949FFF78CFF80
:1024300005F5CA7204F118000649BDE83840FFF7F7
:1024400083BF00BFB42F0020242400204441000893
:102450004C4100085841000870B5044608460D4636
:10246000FEF782FDC6B22046013403780BB9184648
:1024700070BD32462946FEF75FFD0028F3D10120EA
:1024800070BD00002DE9F84F05460C46FEF76CFDC7
:102490002A49C6B22846FFF7DFFF08B10136F6B277
:1024A00027492846FFF7D8FF08B11036F6B2632E49
:1024B0000DD8DFF88890DFF888A0224FDFF88CB0C5
:1024C000DFF88C802E7846B92670BDE8F88F294653
:1024D0002046BDE8F84F01F0ADBD252E29D10722D9
:1024E00049462846FEF728FD40B9D8F80030236059
:1024F000D8F80430636007350834E3E70822514612
:102500002846FEF719FDA0B90F4BA21C13F8011FB6
:1025100009095B45C95D02F8021C197801F00F0139
:1025200002F10202C95D02F8031CEFD1183408352C
:10253000C8E7267001350134C4E700BFE041000858
:1025400058410008F1410008FFE7F11F0BE8F11FB7
:10255000E8410008BFF34F8F044B1A695107FCD1C3
:10256000D3F810215207F8D1704700BF0020005265
:1025700008B50D4B1B78ABB9FFF7ECFF0B4BDA68D6
:10258000D10741BF0A4A5A6002F188325A60D3F833
:102590000C21D20741BF064AC3F8042102F1883258
:1025A000C3F8042108BD00BF1232002000200052F1
:1025B0002301674508B5114B1B78F3B9104B1A6915
:1025C000510742BFDA6842F04002DA60D3F81021C6
:1025D000520742BFD3F80C2142F04002C3F80C214D
:1025E000FFF7B8FF064BDA6842F00102DA60D3F871
:1025F0000C2142F00102C3F80C2108BD1232002068
:10260000002000520F289ABF00F58060400400208F
:10261000704700004FF400307047000010207047F2
:102620000F2808B50BD8FFF7EDFF00F5003302685F
:10263000013204D104308342F9D1012008BD0020C9
:1026400008BD00000F2810B504463FD8FFF782FFF1
:10265000FFF78EFF1E484FF0FF33072C4361C0F891
:1026600014311DD80361FFF775FF230243F02403E3
:10267000C360C36843F08003C36003695A07FCD496
:10268000FFF768FF2046FFF7BDFF4FF4003100F071
:10269000EDF8FFF78FFF2046BDE81040FFF7C0BF01
:1026A000C0F81031FFF756FFA4F108031B0243F0F6
:1026B0002403C0F80C31D0F80C3143F08003C0F88B
:1026C0000C31D0F810315B07FBD4D9E7002010BDE6
:1026D000002000522DE9F84F40EA0203DB060646CF
:1026E000884691464AD1FFF743FFDFF8B0B0454630
:1026F000A9EB050343441F2B04D8FFF75BFF012020
:10270000BDE8F88F204A2148214F06F178439342D3
:10271000204B214A98BF9A4603F1FC0386BF1F460F
:1027200092465846FFF716FF4FF0FF3303603B68B1
:1027300043F002033B6005F11C022B1FA6EB050EC4
:10274000DAF8004014F00504FAD153F8041F4EF8EB
:1027500003109342F4D1BFF34F8FFFF7FBFE4FF00E
:10276000FF3303603B6823F002033B6020222946CD
:10277000304601F04FFC20B1FFF71CFF0020BDE800
:10278000F88F20362035B3E7FFFF0F0014210052E9
:102790000C20005210200052102100521420005230
:1027A00010B5084C237828B153B9FFF7E1FE012397
:1027B000237010BD23B12070BDE81040FFF7FABEB2
:1027C00010BD00BF1232002010B50244064B043980
:1027D000D2B2904200D110BD441C00B253F8200088
:1027E00041F8040FE0B2F4E7504000580F4B30B509
:1027F0001C6F240405D41C6F1C671C6F44F4004438
:102800001C670B4C236843F4807323600244094B1C
:102810000439D2B2904200D130BD441C00B251F80C
:10282000045F43F82050E0B2F4E700BF00440258D0
:10283000004802585040005807B5012201A9002065
:10284000FFF7C2FF019803B05DF804FB13B504461F
:10285000FFF7F2FFA04206D002A9012241F8044D81
:102860000020FFF7C3FF02B010BD00000144BFF31A
:102870004F8F064B884204D3BFF34F8FBFF36F8F48
:102880007047C3F85C022030F4E700BF00ED00E0C1
:10289000034B1B685B0142BF024B01221A70704759
:1028A000D044025813320020014B1878704700BF03
:1028B00013320020064A536823F001035360EFF3FC
:1028C0000983683383F30988002383F311887047F1
:1028D00030EF00E010B5202383F31188104B5B68C4
:1028E00013F4006318D0F1EE103AEFF309844FF0BF
:1028F000807344F84C3C0B4BDB6844F8083CA4F173
:10290000680383F30988FFF7E3FB18B1064B44F82B
:10291000503C10BD054BFAE783F3118810BD00BF92
:1029200000ED00E030EF00E0F1030008F4030008E0
:10293000F0B5BFF34F8FBFF36F8F1D4B0021C3F86E
:102940005012BFF34F8FBFF36F8F5A6942F40032BA
:102950005A61BFF34F8FBFF36F8FC3F88410BFF37B
:102960004F8FD3F88020C2F3C904C2F34E32520114
:10297000A50743F6E07602EA060E284621464EEA0F
:1029800000070139C3F860724F1C00F14040F6D1D6
:10299000203A12F1200FEED1BFF34F8F5A6942F463
:1029A00080325A61BFF34F8FBFF36F8FF0BD00BF0E
:1029B00000ED00E0FEE70000084A094B09498B42A0
:1029C00004D3094A0021934205D3704752F8040FFB
:1029D00043F8040BF3E743F8041BF4E7E043000873
:1029E000603500206035002060350020D0F894303C
:1029F00030B500229D68D0F8904011464FF0FF306E
:102A000004EB421301329542C3F80019C3F81019C0
:102A1000C3F80809C3F8001BC3F8101BC3F8080B60
:102A2000EED24FF00113C4F81C3830BD00EB810327
:102A30002DE9F04FD3F80CE0DEF814404F1CD4F829
:102A400000C03F034FEA41186568D0F89020654503
:102A50000AD3D2F83438012000FA01F123EA010147
:102A6000C2F83418BDE8F08FBEF81060ACEB050377
:102A7000B34228BF334602EB0806D6F81869B6B24F
:102A8000B3EB860F13D8A6683A44A6F1040A994618
:102A90005AF804BFC2F800B0B9F1040F02D9A9F185
:102AA0000409F5E71E442B44A6606360CCE70020D0
:102AB000BDE8F08F890141F02001016103699B06A7
:102AC000FCD4122000F03CBF10B50A4C2046FEF7A3
:102AD000BDFF094BC4F89030084BC4F89430084C43
:102AE0002046FEF7B3FF074BC4F89030064BC4F8FE
:102AF000943010BD14320020000008402842000825
:102B0000B032002000000440344200080378012B5A
:102B100070B505465DD1494BD0F89040984259D1E7
:102B2000474BD3F8D82042F00062C3F8D820D3F83E
:102B3000002142F00062C3F80021D3F80021D3F84D
:102B4000802042F00062C3F88020D3F8802022F079
:102B50000062C3F88020D3F880300E216520FEF794
:102B6000F3FB384BE360384BC4F800380023C4F85B
:102B7000003EC0232360D5F890604FF40413A36394
:102B80003369002BFCDA012333610C2000F0D8FEFE
:102B90003369DB07FCD4122000F0D2FE3369002B2E
:102BA000FCDA0026A6602846FFF720FF6B68C4F811
:102BB0001068DB68C4F81468C4F81C68002B3AD1AC
:102BC000224BA3614FF0FF336361A36843F001031D
:102BD000A36070BD1E4B9842C8D1194BD3F8D820C2
:102BE00042F00072C3F8D820D3F8002142F00072FE
:102BF000C3F80021D3F80021D3F8802042F00072FE
:102C0000C3F88020D3F8802022F00072C3F880201F
:102C1000D3F88020D3F8D82022F08062C3F8D820DF
:102C2000D3F8002122F08062C3F80021D3F80031EC
:102C30000E214D2093E7074BC3E700BF143200205D
:102C4000004402584014004003002002003C30C001
:102C5000B0320020083C30C0F8B5D0F890400546AE
:102C600000212046FFF726FFD5F8941000234FF0EF
:102C700001128F68C4F834384FF00066C4F81C287D
:102C80004FF0FF3004EB431201339F42C2F800695A
:102C9000C2F8006BC2F80809C2F8080BF2D20B6840
:102CA000D5F89020C5F89830636210231361166937
:102CB00016F01006FBD1122000F042FED4F80038C6
:102CC00023F4FE63C4F80038A36943F4402343F0BF
:102CD0001003A3610923C4F81038C4F814380B4B4F
:102CE000EB604FF0C043C4F8103B094BC4F8003B05
:102CF000C4F81069C4F80039D5F8983003F110020F
:102D000043F48013C5F89820A362F8BD044200087C
:102D100040800010D0F8902090F88A10D2F8003847
:102D200023F4FE6343EA0113C2F800387047000041
:102D30002DE9F0410EB200EB86080D46D8F80C10D4
:102D40000F6807F00303022B53D0032B53D03F4AE5
:102D50003F4F012B18BF1746D0F890404FEA451E51
:102D600004EB0E030022C3F8102B8A6905F1100C46
:102D7000002A42D04A8A05F158035B013A43E250E7
:102D80000123D4F81C2803FA0CF31343A6444A6920
:102D9000C4F81C380023CEF8103905F13F03002A8F
:102DA0003BD00A8A898B9208012988BF4A43D0F810
:102DB000981004EB8303561841EA0242C0F8986069
:102DC00029465A602046FFF775FED8F80C301B8A5A
:102DD00043EA85531F4305F148035B01E750012394
:102DE000D4F81C2803FA05F51543C4F81C58BDE8AF
:102DF000F081184FB0E7184FAEE704EB4613D3F855
:102E0000002B22F40042C3F8002BD4F81C28012325
:102E100003FA0CF322EA0303B8E704EB83030F4A37
:102E20005A6004EB461629462046FFF743FED6F8C3
:102E3000003923F40043C6F80039D4F81C380122C5
:102E400002FA05F523EA0505CFE700BF0080001070
:102E5000008004100080081000800C1000040002A4
:102E6000D0F894201268C0F89820FFF7BFBD00008A
:102E70005831D0F8903049015B5813F4004004D029
:102E800013F4001F14BF0120022070474831D0F80E
:102E9000903049015B5813F4004004D013F4001F34
:102EA00014BF01200220704700EB8101CB68196A32
:102EB0000B6813604B6853607047000000EB8103A0
:102EC00030B5DD68AA691368D36019B9402B84BF97
:102ED000402313606B8A1468D0F890201C44013C96
:102EE000B4FBF3F46343033323F0030302EB411019
:102EF00043EAC44343F0C043C0F8103B2B6803F0DF
:102F00000303012B09B20ED1D2F8083802EB4110AD
:102F100013F4807FD0F8003B14BF43F0805343F09C
:102F20000053C0F8003B02EB4112D2F8003B43F0E3
:102F30000443C2F8003B30BD2DE9F041D0F8906069
:102F400006EB41130546D3F8087BC3F8087B3A0724
:102F50000C4608D5D6F814381B0704D500EB8103BE
:102F6000DB685B689847FA072FD5D6F81438DB077B
:102F70002BD505EB8403D968CCB98B69488A5E6888
:102F8000B6FBF0F200FB12628AB91868DA68904268
:102F90000DD2121A83E81400202383F311882146EE
:102FA0002846FFF78BFF84F31188BDE8F0810123E9
:102FB00003FA04F26B8923EA02036B81CB6823B125
:102FC00021462846BDE8F0411847BDE8F0810000E1
:102FD00000EB810370B5DD68D0F890306C6926682D
:102FE000E6604A0156BB1A444FF40020C2F81009AB
:102FF0002A6802F00302012A0AB20ED1D3F80808A7
:1030000003EB421410F4807FD4F8000914BF40F0A1
:10301000805040F00050C4F8000903EB4212D2F88F
:10302000000940F00440C2F80009D3F83408012236
:1030300002FA01F10143C3F8341870BD19B9402EEA
:1030400084BF4020206020682E8A841940F0005000
:10305000013C1A44B4FBF6F440EAC440C6E7000061
:103060002DE9F041D0F8906006EB41130446D3F807
:103070000879C3F80879FB070D461CD5D6F8103837
:10308000DA0718D500EB8103D3F80CE0DEF8143032
:10309000D3F800C0DA6894451BD2A2EB0C024FF0C3
:1030A00000081A60C3F80480202383F31188FFF717
:1030B0008FFF88F311883B0618D5D6F834280123F2
:1030C000AB40134212D029462046BDE8F041FFF73D
:1030D000ADBC012303FA01F2038923EA0203038151
:1030E000DEF80830002BE6D09847E4E7BDE8F08131
:1030F0002DE9F047D0F890506E69AB691E40F1049D
:1031000004466E6103D5BDE8F047FEF719BD002EF9
:1031100011DAD5F8003E9A071EBFD5F8003E23F01D
:103120000303C5F8003ED5F8043823F00103C5F8C1
:103130000438FEF735FD330502D52046FEF724FDA1
:10314000B7040CD5D5F8083813F0060FEB6823F454
:1031500070530CBF43F4105343F4A053EB6030079B
:1031600004D56368DB680BB120469847F10200F193
:10317000A180B2020BD5D4F8908000274FF001094E
:10318000D4F894309B68F9B28B4280F0D280F30679
:103190001AD5D4F890100A6AC2F30A1702F00F0386
:1031A00002F4F012B2F5802F00F0EC80B2F5402F5F
:1031B0000AD104EB830301F58051DB68186A002310
:1031C0001A469F4240F0D1803003D5F8185835D5C3
:1031D000E90303D500212046FFF7AEFEAA0303D57D
:1031E00001212046FFF7A8FE6B0303D502212046EC
:1031F000FFF7A2FE2F0303D503212046FFF79CFE15
:10320000E80203D504212046FFF796FEA90203D564
:1032100005212046FFF790FE6A0203D506212046CD
:10322000FFF78AFE2B0203D507212046FFF784FE15
:10323000EF0103D508212046FFF77EFE700340F121
:10324000C980E90703D500212046FFF709FFAA0737
:1032500003D501212046FFF703FF6B0703D50221A9
:103260002046FFF7FDFE2F0703D503212046FFF779
:10327000F7FEEE0603D504212046FFF7F1FEA8066F
:1032800003D505212046FFF7EBFE690603D506218D
:103290002046FFF7E5FE2A0603D507212046FFF763
:1032A000DFFEEB0540F1968020460821BDE8F0479F
:1032B000FFF7D6BED4F890904FF000084FF0010A07
:1032C000D4F894309B685FFA88F7BB42FFF451AFA3
:1032D00009EB4713D3F8002902F44022B2F5802FFE
:1032E00024D1D3F80029002A20DAD3F8002942F0AB
:1032F0009042C3F80029D3F80029002AFBDB3946A5
:10330000D4F89000FFF7D6FB22890AFA07F322EAE5
:103310000303238104EB8703DB689B6813B1394601
:103320002046984739462046FFF780FB08F1010800
:10333000C6E708EB4112D2F8003B03F44023B3F593
:10334000802F10D1D2F8003B002B0CDA628909FAE9
:1033500001F322EA0303638104EB8103DB68DB688A
:103360000BB12046984701370AE713F0030F08BF57
:103370000A68072B98BF027003F101039CBF120A71
:1033800001301EE704EB830301F58051DA68906990
:103390000268D0F808C04068A2EB000E0022104678
:1033A000974208D1DB689B699A683A449A605A68E8
:1033B00017445F6008E712F0030F08BF08689645DE
:1033C00088BF8CF8000002F1010284BF000A0CF1F2
:1033D000010CE5E7BDE8F08708B50348FFF788FE74
:1033E000BDE80840FFF776BA1432002008B503485C
:1033F000FFF77EFEBDE80840FFF76CBAB032002050
:10340000D0F8903003EB4111D1F8003B43F40013A6
:10341000C1F8003B70470000D0F8903003EB411139
:10342000D1F8003943F40013C1F8003970470000A7
:10343000D0F8903003EB4111D1F8003B23F4001396
:10344000C1F8003B70470000D0F8903003EB411109
:10345000D1F8003923F40013C1F800397047000097
:1034600030B5039C0172043304FB0325C361049B44
:1034700003630021059B00604060C16042610261FE
:103480008561046242628162C162436330BD0000B3
:103490000022416A41610161C2608262C2626FF0D2
:1034A0000101FEF79DBE000003694269934203D10A
:1034B000C2680AB100207047181D7047036919607F
:1034C000C2680132C260C2691344826903619342D7
:1034D00024BF436A03610021FEF776BE38B5044677
:1034E0000D46E3683BB16269131D1268A362134481
:1034F000E362002038BD237A33B929462046FEF71F
:1035000053FE0028EDDA38BD6FF00100FBE7000044
:10351000C368C269013BC360436913448269436164
:10352000934224BF436A436100238362036B03B168
:103530001847704770B52023044683F31188866AC4
:103540003EB9FFF7CBFF054618B186F31188284630
:1035500070BDA36AE26A13F8015BA362934202D3CF
:103560002046FFF7D5FF002383F31188EFE7000023
:103570002DE9F84F04460E4690469946202787F3DA
:1035800011880025AA46D4F828B0BBF1000F09D154
:1035900049462046FFF7A2FF20B18BF31188284649
:1035A000BDE8F88FA16AE36AA8EB050B5B1A9B459F
:1035B00028BF9B46BBF1400F1BD9334601F14002A7
:1035C00051F8040B43F8040B9142F9D1A36A40333C
:1035D0004036A3624035A26AE36A9A4202D320468B
:1035E000FFF796FF8AF311884545D8D287F31188F3
:1035F000C9E730465A46FDF795FCA36A5B445E4432
:10360000A3625D44E7E7000010B5029C0172043339
:1036100003FB0421C36100238362C362039B036332
:10362000049B00604060C460426102618161046289
:103630004262436310BD0000026AC260426A426196
:10364000026100228262C2626FF00101FEF7C8BD12
:10365000436902699A4203D1C2680AB100207047E7
:10366000184650F8043B0B6070470000C368C269FD
:103670000133C3604369134482694361934224BFA9
:10368000436A43610021FEF79FBD000038B5044640
:103690000D46E3683BB123691A1DA262E269134437
:1036A000E362002038BD237A33B929462046FEF76D
:1036B0007BFD0028EDDA38BD6FF00100FBE700006C
:1036C00003691960C268013AC260C2691344826921
:1036D0000361934224BF436A036100238362036B47
:1036E00003B118477047000070B5202304460E460A
:1036F00083F31188856A35B91146FFF7C7FF10B10A
:1037000085F3118870BDA36A1E70A36AE26A013353
:103710009342A36204D3E16920460439FFF7D0FF46
:10372000002080F3118870BD2DE9F84F04460D4646
:1037300091469A464FF0200888F311880026B34638
:10374000A76A4FB951462046FFF7A0FF20B187F383
:1037500011883046BDE8F88FA06AE76AA9EB060336
:103760003F1A9F4228BF1F46402F1BD905F1400337
:1037700055F8042B40F8042B9D42F9D1A36A40333D
:10378000A3624036A26AE36A9A4204D3E169204602
:103790000439FFF795FF8BF311884E45D9D288F392
:1037A0001188CDE729463A46FDF7BCFBA36A3B44A6
:1037B0003D44A3623E44E5E7026943699A4203D16E
:1037C000C3681BB9184670470023FBE7836A002BC8
:1037D000F8D0043B9B1AF5D01360C368013BC3606B
:1037E000C3691A44836902619A4224BF436A036130
:1037F000002383620123E5E700F052B9034B002266
:1038000058631A610222DA60704700BF000C004062
:10381000014B0022DA607047000C0040014B5863F6
:10382000704700BF000C0040FEE7000010B5194CC7
:10383000FEF7C0FBFEF7E2FC802217492046FEF7A8
:1038400067FC012344F8180C0374144B144AD9681C
:1038500021F4E0610904090C0A431249DA60CA68DC
:1038600042F08072CA60104A1049C2F8B01F116855
:1038700041F0010111601022DA77202283F8222022
:10388000002383F3118862B60948BDE81040FEF7B3
:1038900061BC00BFD42A00204042000800ED00E0D7
:1038A0000003FA05F0ED00E0001000E055CEACC5D5
:1038B000484200082DE9F84F1F4CDFF880906569F9
:1038C00004F114074FF00008D9F82430266AAA68DA
:1038D0009E1B96421DD34FF0200AAA68236AD5F892
:1038E0000CB0134423622B68BB425F60A6EB020658
:1038F0006361C5F80C8001D1FFF78AFF88F3118856
:103900002869D8478AF311886569AB689E42E4D27A
:10391000DAE76269BA420CD0916823628E1B966026
:10392000A86802282CBF1818981CBDE8F84FFFF7AC
:1039300075BFBDE8F88F00BFAC2A0020000C004026
:10394000034B59685A68521A9042FBD8704700BF1F
:10395000001000E04B6843608B688360CB68C360F5
:103960000B6943614B6903628B6943620B680360B7
:103970007047000008B52C4B2C48D3F8882040F243
:10398000FF710A43C3F88820D3F8882022F4FF622D
:1039900022F00702C3F88820D3F88820D3F8E0206B
:1039A0000A43C3F8E020D3F808210A43C3F80821EA
:1039B0001F4AD3F808311146FFF7CCFF1D4802F12A
:1039C0001C01FFF7C7FF1C4802F13801FFF7C2FFD7
:1039D0001A4802F15401FFF7BDFF194802F17001C6
:1039E000FFF7B8FF174802F18C01FFF7B3FF164845
:1039F00002F1A801FFF7AEFF144802F1C401FFF77E
:103A0000A9FF134802F1E001FFF7A4FF114802F1FA
:103A1000FC01FFF79FFF104802F58C71FFF79AFF3A
:103A2000BDE8084000F016B90044025800000258F2
:103A3000684200080004025800080258000C0258AE
:103A4000001002580014025800180258001C0258B6
:103A500000200258002402580028025808B500F03F
:103A6000C7FAFFF7E3FEFEF713FFBDE80840FEF7D5
:103A7000CFBC000070470000084B1A69920710B5D0
:103A800008D500241C61202383F31188FFF712FF5F
:103A900084F31188BDE81040FEF71CBF000C004005
:103AA000124BD3F8E82042F00802C3F8E820D3F81C
:103AB000102142F00802C3F810210D4AD3F810314A
:103AC000D36B43F00803D3630A4B63229A624FF02F
:103AD000FF32DA6200229A615A63DA605A60012288
:103AE0005A6108211A603220FDF72EBC00440258AA
:103AF0000010005C000C0040F8B5514BD3F880205A
:103B00004FF0FF32C3F880200024D3F88010C3F8B0
:103B10008040D3F88010D3F88410C3F88420D3F801
:103B20008410C3F88440D3F88410D96F41F0FF416A
:103B300041F4FF0141F4DF4141F07F01D967D96FC2
:103B400021F0FF4121F4FF0121F4DF4121F07F0149
:103B5000D967D96FD3F888106FEA41516FEA515194
:103B6000C3F88810D3F88810C1F30A01C3F888108D
:103B7000D3F88810D3F89010C3F89020D3F89010A1
:103B8000C3F89040D3F89010D3F89410C3F8942061
:103B9000D3F89410C3F89440D3F89410D3F8981045
:103BA000C3F89820D3F89810C3F89840D3F8981029
:103BB000D3F88C10C3F88C20D3F88C10C3F88C4049
:103BC000D3F88C10D3F89C10C3F89C20D3F89C2019
:103BD000C3F89C40D3F89C3000F0EAF9194B072257
:103BE0009A60194ADA60194A1A6105225A60184A1D
:103BF000536A43F480335362C2F88440BFF34F8F5B
:103C0000D2F88030C3F3C904C3F34E335B01A50778
:103C100043F6E07603EA060E284621464EEA000700
:103C20000139C2F874724F1C00F14040F6D1203BBC
:103C300013F1200FEED1BFF34F8FBFF36F8FF8BD9D
:103C40000044025890ED00E0000004301B0008031F
:103C500000ED00E05A4B5B4901221A605A4B196093
:103C60009A605A4ADA6000221A614FF440429A611F
:103C70009A699204FCD51A6842F480721A60544B17
:103C80001A6F12F4407F1FBF4FF480321A67002270
:103C90001A671A6842F001021A604D4A1346116809
:103CA0004807FCD5002111611A6912F03802FBD1D6
:103CB000012119604FF0804159605A67454ADA6224
:103CC000454A1A611A6842F480321A60404A134623
:103CD00011688903FCD5116841F0800111601A68F0
:103CE000D205FCD53D4A3E499A6200225A631963C7
:103CF000A1F5C0214B39DA6399635A64394A1A64D1
:103D0000394ADA621A6842F0A8521A60304B1A68CF
:103D100002F02852B2F1285FF9D109229A610022FB
:103D2000DA611A624FF00052DA643049304A1A659B
:103D300059659A652F4A212111601A6942F00302E0
:103D40001A61234B1A6902F03802182AFAD1D3F803
:103D5000DC2042F00052C3F8DC20D3F8042142F00A
:103D60000052C3F80421D3F80421D3F8DC2042F038
:103D70008042C3F8DC20D3F8042142F08042C3F82B
:103D80000421D3F80421D3F8DC2042F00042C3F828
:103D9000DC20D3F8042142F00042C3F80421D3F818
:103DA0000421D3F8F42042F00202C3F8F420D3F83F
:103DB0001C2142F00202C3F81C21D3F81C317047C9
:103DC0000881005100C000F00048025802000001C4
:103DD000004402580000FF010088900822204000A3
:103DE0006302070147040508FD0BFF010010E00016
:103DF0000000011000200052084A08B593681168BD
:103E00000B4003F00103936023B1054A13680BB123
:103E100050689847BDE80840FEF75CBD8000005838
:103E2000C0250020084A08B5936811680B4003F0CC
:103E30000203936023B1054A93680BB1D068984799
:103E4000BDE80840FEF746BD80000058C0250020B0
:103E5000084A08B5936811680B4003F004039360A7
:103E600023B1054A13690BB150699847BDE8084072
:103E7000FEF730BD80000058C0250020084A08B574
:103E8000936811680B4003F00803936023B1054A5F
:103E900093690BB1D0699847BDE80840FEF71ABD99
:103EA00080000058C0250020084A08B593681168B2
:103EB0000B4003F01003936023B1054A136A0BB162
:103EC000506A9847BDE80840FEF704BD80000058DE
:103ED000C0250020174B10B59C681A68144004F4E4
:103EE00078729A60A30604D5134A936A0BB1D06A1C
:103EF0009847600604D5104A136B0BB1506B984776
:103F0000210604D50C4A936B0BB1D06B9847E205A0
:103F100004D5094A136C0BB1506C9847A30504D51E
:103F2000054A936C0BB1D06C9847BDE81040FEF782
:103F3000D1BC00BF80000058C02500201A4B10B52E
:103F40009C681A68144004F47C429A60620504D5A7
:103F5000164A136D0BB1506D9847230504D5134ACB
:103F6000936D0BB1D06D9847E00404D50F4A136EE2
:103F70000BB1506E9847A10404D50C4A936E0BB157
:103F8000D06E9847620404D5084A136F0BB1506F86
:103F90009847230404D5054A936F0BB1D06F984717
:103FA000BDE81040FEF796BC80000058C0250020F8
:103FB000062108B50846FDF7C7F906210720FDF7D9
:103FC000C3F906210820FDF7BFF906210920FDF7F6
:103FD000BBF906210A20FDF7B7F906211720FDF7E6
:103FE000B3F906212820BDE80840FDF7ADB900006F
:103FF00008B5FFF781FDFDF77FF8FDF74BFBFDF7F7
:1040000023FDFDF7F5FBFFF735FDBDE80840FFF7A1
:10401000F3BB000010B501390244904201D10020E9
:1040200010BD10F8013B11F8014FA342F5D0181B49
:1040300010BD0000034611F8012B03F8012B002AE4
:10404000F9D17047121012131211000001105A001A
:10405000031059000120580003205600EC2A0020CC
:104060004026002053544D333248373F3F3F0053E2
:10407000544D3332483734332F3735330000000086
:10408000009600000000000000000000000000009A
:104090000000000000000000000000005D160008A5
:1040A0004916000885160008711600087D160008DC
:1040B00069160008551600084116000891160008F8
:1040C0000000000069170008551700089117000844
:1040D0007D17000889170008751700086117000888
:1040E0004D170008ED170008000000000100000057
:1040F0000000000002000000000000009519000808
:10410000011A000840004000842F0020942F002056
:10411000020000000000000003000000000000009A
:10412000451A00080000000010000000A42F002025
:104130000000000001000000000000001432002018
:1041400001010200486F6C7962726F004475726100
:104150006E64616C2D424C002553455249414C25FB
:1041600000000000B123000819230008011900080D
:1041700095230008430000007C4100080902430029
:10418000020100C0320904000001020201000524FE
:104190000010010524010001042402020524060088
:1041A00001070582030800FF09040100020A00005C
:1041B00000070501024000000705810240000000E1
:1041C00012000000C8410008120110010200004066
:1041D00062314B00000201020301000004030904E4
:1041E00025424F4152442500447572616E64616CF2
:1041F0000030313233343536373839414243444563
:104200004600000000000000B51B0008951E0008D5
:10421000411F0008400040004C3300204C33002078
:10422000010000005C33002080000000400100001D
:104230000800000000010000000400000800000069
:104240006D61696E00000000604200086833002064
:10425000603500200100000029380008000000003F
:1042600069646C65000000000000802A0000000006
:10427000AAAAAAAA00000000FFFF00000000000098
:1042800000A00A000400000000000000AAAAAAAAD8
:1042900000000000FDFF0000000000000000000022
:1042A0000050000000000000AAAAAAAA0000000016
:1042B0003FFF0000000000000000000000000000C0
:1042C00000000000AAAAAAAA00000000FFFF000048
:1042D00000000000000000000000020000000000DC
:1042E000AAAAAAAA00000100FFFF00000000000027
:1042F000070000000020000000000000AAAAAAAAEF
:1043000000100000FFFF0000000000070000000098
:104310000000000000000000AAAAAAAA00000000F5
:10432000FFFF00000000000000000000000000008F
:1043300000000000AAAAAAAA00000000FFFF0000D7
:10434000000000000000000000000000000000006D
:10435000AAAAAAAA00000000FFFF000000000000B7
:10436000000000000000000000000000AAAAAAAAA5
:1043700000000000FFFF000000000000000000003F
:104380000000000000000000AAAAAAAA0000000085
:10439000FFFF00000000000000000000000000001F
:1043A000FF00000000000000644000083F00000023
:1043B000500400006F4000083F000000009600001D
:1043C0000000080004000000DC41000800000000BC
:1043D00000000000000000000000000000000000DD
:0443E00000000000D9
:00000001FF
